:100000000C9417060C943E290C946B290C943F0613
:100010000C943F060C943F060C943F060C943F064C
:100020000C943F060C943F060C94BA0C0C943F06BB
:100030000C943F060C943F060C943F060C943F062C
:100040000C9498290C943F060C94522D0C948D2DF1
:100050000C943F060C943F060C943F060C943F060C
:100060000C943F060C943F068F1C961C961C8F1C0C
:10007000961C961C961C961C961C961C961C961CF0
:10008000961C961C961C961C961C041C961C961C72
:10009000961C961C961C671B961C961C961C961C00
:1000A000961C961C961C961C961C961C961C961CC0
:1000B000961C961C961C101C101C101C101C101C4E
:1000C000101C101C101C101C961C961C961C961CB8
:1000D000961C961C6C1B0F1C0F1C0F1C0F1C961CD7
:1000E000201C281C301C381C401C481C501C581C50
:1000F000621C6C1C761C801CB31B731B961C961C0C
:10010000961C961C041C961C961C961C961C961CF1
:10011000961C961C961C0E1C0E1C0E1C0E1C961C6F
:10012000201C281C301C381C401C481C501C581C0F
:10013000621C6C1C761C801CB31B731B961C961CCB
:10014000961C961C041CC71CC71CC71CC71CC71CBC
:10015000C71CC71CC71CC71CC71CC71CC71CC71C87
:10016000E71DE71DE71DE71DE71DE71D0E1D181D17
:10017000221D2C1D921D9C1DAA1DBB1D581EC81E94
:10018000991E9E1EA31EA81EAD1EB21EB71EC81E1F
:10019000C21ECD25E225EE25F72504262A26322685
:1001A00055264226456E746572206D656E752E2E3D
:1001B0002E00546F67676C6564206D6963726F50C1
:1001C000504D00546F67676C656420696E76657288
:1001D0007465642050504D2100546F67676C6564EE
:1001E000205458206D7574696E672100546F6767DD
:1001F0006C65642074656C656D657472792100505E
:10020000726F746F636F6C206572726F72207769A2
:1002100074682052580054696D656F757420776852
:10022000656E20636F6E6E656374696E6720746FB0
:1002300020525800507265737320616E79206B658F
:100240007920746F2063616E63656C00436F6E6E1E
:10025000656374696E6720746F2052582C20706F2C
:100260007765722075702074686520525820287751
:100270006974682062696E6420706C7567206966B5
:10028000206E6F74207573696E6720616C77617979
:10029000732062696E642900546F67676C6564201F
:1002A00027696D6D656469617465206F757470751B
:1002B000742700546F67676C65642027736C6176E0
:1002C00065206D6F64652700546F67676C656420F7
:1002D00027616C776179732062696E642700546FBF
:1002E00067676C65642050504D206368616E6E6571
:1002F0006C206C696D6974005365742052535349C6
:1003000020696E6A656374696F6E206368616E6EE2
:10031000656C2028303D3D64697361626C6529001D
:100320005365742050504D206D696E696D756D2058
:1003300073796E630053657420626561636F6E202C
:10034000696E74657276616C0053657420626561D4
:10035000636F6E2064656C6179005365742062651B
:1003600061636F6E206672657175656E6379206971
:100370006E20487A3A20303D64697361626C652C66
:100380002050783D504D52206368616E6E656C2040
:10039000782C2046783D465253206368616E6E6526
:1003A0006C2078005365742050574D2073746F7023
:1003B0002064656C61792028302064697361626C07
:1003C00065642C20312D323535203D3D20302E31D5
:1003D00073202D2035306D696E29005365742050CF
:1003E000504D2073746F702064656C6179202830E3
:1003F0002064697361626C65642C20312D3235355F
:10040000203D3D20302E3173202D2035306D696E1A
:100410002900536574206661696C736166652064A8
:10042000656C61792028302064697361626C656451
:100430002C20312D323535203D3D20302E3173209A
:100440002D2035306D696E29002A2A2A2A2A2A2A67
:100450002A2A2A2A2A2A2A2A2A2A2A2A2A2A2A2AFC
:100460002A2A2A2A2A2A0052582041636B656420CE
:100470002D2072657665727420737563636573737E
:1004800066756C21002A2A2A2A2A2A2A2A2A2A2A36
:100490002A2A2A2A2A2A2A2A2A2A2A2A2A2A2A2ABC
:1004A0002A2A002A2A2A2A2A2A2A2A2A2A2A2A2AD6
:1004B0002A2A2A2A2A2A2A2A2A2A2A2A2A2A2A2A9C
:1004C0000052582041636B6564202D207570646173
:1004D0007465207375636365737366756C21002A98
:1004E0002A2A2A2A2A2A2A2A2A2A2A2A2A2A2A2A6C
:1004F0002A2A2A2A2A2A2A2A2A2A2A2A0056616CE1
:1005000069642063686F69636573206172653A206E
:100510005B315D2D5B31365D20286368616E6E65F1
:100520006C20312D31362900536574206F7574703D
:10053000757420666F7220706F727420005B585D56
:100540002061626F7274206368616E6765732061F9
:100550006E64206578697420525820636F6E6669F6
:1005600067005B535D207361766520736574746901
:100570006E677320746F205258005B525D20726565
:10058000766572742052582073657474696E67734F
:1005900020746F2064656661756C747300557365B3
:1005A000206E756D62657273205B312D445D207421
:1005B0006F206564697420706F727473205B452DC1
:1005C000515D20666F722073657474696E67730085
:1005D000202D20726563656976657220636F6E6693
:1005E0006967757261746F722C207278207377203E
:1005F000000A0A6F70656E4C52536E672000536597
:10060000742073657269616C2062617564726174D3
:10061000653A200056616C69642063686F696365A0
:10062000733A2031202D20342B34202F2032202DDE
:100630002038202F2033202D20382B34202F203419
:10064000202D203132202F2035202D2031322B3407
:10065000202F2036202D203136005365742043682A
:10066000616E6E656C20636F6E6669673A20005339
:1006700065742044617461726174652028302D3284
:10068000293A200053657420486F70206368616EBA
:100690006E656C7320286D61782032342C20736570
:1006A0007061726174656420627920636F6D6D6141
:1006B00073292076616C69642076616C756573209E
:1006C000312D3235353A2000536574206368616EF0
:1006D0006E656C2073706163696E672028783130B5
:1006E0006B487A293A200053657420524620706F77
:1006F0007765722028302D37293A20005365742001
:100700005246206D616769632028686578292065F5
:100710002E672E20307844454144463030443A20FC
:10072000005365742062617365206672657175653A
:100730006E63792028696E20487A293A20005B5A36
:100740005D20656E74657220726563656976657299
:1007500020636F6E66696775726174696F6E20756C
:1007600074696C79005B465D20646973706C6179B3
:100770002061637475616C206672657175656E6366
:100780006965732075736564005B525D2063616CFD
:1007900063756C6174652072616E646F6D206B654A
:1007A0007920616E6420686F70206C697374005BDF
:1007B000495D207265696E697469616C697A65204A
:1007C00073657474696E677320746F20736B6574DE
:1007D00063682064656661756C7473005B585D20A6
:1007E000726576657274206368616E6765732061F7
:1007F0006E642065786974206D656E75005B535D6D
:1008000020736176652073657474696E67732074F4
:100810006F20454550524F4D20616E6420657869C8
:1008200074206D656E7500557365206E756D62651B
:100830007273205B302D395D20746F20656469749C
:1008400020706172616D657465727300202D205394
:10085000797374656D20636F6E6669677572617414
:10086000696F6E000A0A6F70656E4C52536E672096
:10087000005129204F7574707574206265666F721F
:1008800065206C696E6B20283D465329203A200074
:10089000502920536C617665206D6F646520286552
:1008A00078706572696D656E74616C293A20004FCD
:1008B000292054696D65642042494E4420617420AA
:1008C0007374617274757020203A20004E29205094
:1008D000504D206F7574707574206C696D69746506
:1008E0006420202020203A200044495341424C45B6
:1008F00044004D292050504D205253534920746FCD
:10090000206368616E6E656C202020203A20004CC8
:10091000292050504D206D696E696D756D20737979
:100920006E63202875732920203A200044495341E2
:10093000424C4544004B29204661696C73616665F1
:1009400020626561636F6E20696E74762E20283197
:100950002D32353573293A20004A29204661696CC9
:100960007361666520626561636F6E2064656C61AA
:10097000792028302D323535203D3E20313073200E
:100980002D203135306D696E293A200049292046E5
:1009900061696C7361666520626561636F6E206674
:1009A00072712E203A200048292050574D20737430
:1009B0006F702064656C6179202020202020203A0F
:1009C000200047292050504D2073746F70206465BB
:1009D0006C6179202020202020203A200046292008
:1009E0004661696C736166652064656C617920207D
:1009F00020202020203A200050574D206368616E4F
:100A00006E656C200066756E6374696F6E3A2000C7
:100A10002920706F72742000506F776572546F7761
:100A2000657200445446205548462033322D626991
:100A3000742031306368004F70656E4C52536E679E
:100A40005258206D696E6920342F36636800466CF9
:100A50007974726F6E2F4F72616E676552582055B0
:100A600048462038636800525820747970653A20EF
:100A70000044697361626C656400487A00203D3D02
:100A8000200043616C63756C617465642070616300
:100A90006B657420696E74657276616C3A200042F1
:100AA00029204D6963726F202868616C6629205087
:100AB000504D202020203A00412920496E76657251
:100AC0007465642050504D20696E20202020203A0B
:100AD000003029204D7574652062757A7A65722020
:100AE000286D6F73746C79293A0039292053657227
:100AF00069616C2062617564726174653A00736D3E
:100B0000617274506F7274004672536B7900547244
:100B1000616E73706172656E740044697361626CBA
:100B200065640038292054656C656D657472793A86
:100B300020202020202020003729204368616E6E6D
:100B4000656C20636F6E6669673A20200036292045
:100B500044617461726174652028302D32293A2015
:100B6000202000352920486F70206368616E6E6513
:100B70006C733A2020202020003429204368616EC5
:100B80006E656C2073706163696E673A2020003374
:100B90002920524620706F7765722028302D372922
:100BA0003A202020003229205246206D6167696377
:100BB0003A202020202020202020003129204261BE
:100BC0007365206672657175656E63793A202020C1
:100BD0000000000000240027002A0000000000257B
:100BE0000028002B0000000000230026002900043C
:100BF00004040404040404020202020202030303C4
:100C000003030301020408102040800102040810BD
:100C1000200102040810200000000700020100006B
:100C2000030406000000000000000000352F11241E
:100C30001FBECFEFD8E0DEBFCDBF13E0A0E0B1E034
:100C4000ECEAF0E602C005900D92A839B107D9F799
:100C500016E0A8E9B3E001C01D92AB35B107E1F79A
:100C60001CE0CEE2DCE004C02297FE010E9431309D
:100C7000CC32D107C9F70E947A2F0C9454300C94CF
:100C80000000A0E0B0E0E7E4F6E00C940030EC01F6
:100C9000A880B980CA80DB80A114B104C104D1044A
:100CA00041F484E2A82E89EDB82E8BE5C82E87E0AA
:100CB000D82EC601B5012DE133EF41E050E00E948E
:100CC000DD2F27EA31E440E050E00E94892F7B01CC
:100CD0008C01C601B5012DE133EF41E050E00E94E7
:100CE000DD2FCA01B9012CEE34EF4FEF5FEF0E9408
:100CF000892F6E0D7F1D801F911F97FF04C06150CB
:100D0000704080409048688379838A839B839B01ED
:100D1000AC015F77B901CA01CDB7DEB7EAE00C9448
:100D20001C300E944106089581EB92E00E9441062A
:100D300008956093B1027093B2028093B3029093CE
:100D4000B4020895A0E0B0E0E8EAF6E00C94F92FD0
:100D5000EC012B016A016115710519F0FB0191830A
:100D60008083C114D10449F0C6010297839728F00B
:100D700020E030E040E050E0DCC0A9908A2D90E017
:100D80000E944930892BC9F7FDE2AF1621F4A990E2
:100D90003324339405C08BE2A81609F4A9903324B8
:100DA000C114D10421F0E0E1CE16D10411F5F0E335
:100DB000AF1669F48881883711F0883541F4A9802D
:100DC000229682E0382A20E1C22ED12C12C0C11412
:100DD000D10479F4E0E3AE1659F199E9E92E99E9E5
:100DE000F92E99E9092F99E1192F8AE0C82ED12C03
:100DF0003AC0FAE0CF16D10491F080E1C816D104D0
:100E000029F0E8E0CE16D104F9F415C0BFEFEB2EBF
:100E1000BFEFFB2EBFEF0B2FBFE01B2F24C0A9E9B4
:100E2000EA2EA9E9FA2EA9E90A2FA9E11A2F1BC077
:100E3000F8E0CF2ED12CEFEFEE2EEFEFFE2EEFEFFE
:100E40000E2FEFE11E2F0FC09601442737FD40956E
:100E5000542F6FEF7FEF8FEF9FEF0E94BB2FC901E1
:100E6000DA017C018D0120E030E040E050E060E0FC
:100E70003601882477FC8094982C70EDB72EBA0C3C
:100E8000F9E0FB1570F48A2D81548A3118F499EC3D
:100E9000B92E06C08A2D81568A3148F589EAB82EC6
:100EA000BA0C8B2D90E08C159D050CF56F3FE9F089
:100EB000E216F30604071507B8F0CA01B901A40148
:100EC00093010E94892F9B01AC018B2D90E0A0E043
:100ED000B0E0280F391F4A1F5B1F281739074A0740
:100EE0005B0710F061E001C06FEFA990C6CF41141D
:100EF000510451F0662311F0219703C031FE04C064
:100F00002297F201D183C08330FE07C050954095EF
:100F1000309521953F4F4F4F5F4F67FF0AC082E2E8
:100F200090E090935A06809359062FEF3FEF4FEFD2
:100F30005FEFB901CA01CDB7DEB7E1E10C9415301E
:100F4000FC0188279927E89421912032E9F3293080
:100F500010F02E30C8F32B3241F02D3239F4689462
:100F600004C00E94F507820F911D219120532A3061
:100F7000C0F31EF4909581959F4F089548E953E082
:100F80000E94C3070895009731F4DA018D919C9176
:100F9000009709F40EC0DC01FB013D912191222351
:100FA00019F03217C9F3FACF332331F4DA011D9265
:100FB0001C928827992708951197AF93BF93FB013F
:100FC0003D912191321771F4332321F48827992719
:100FD000119702C01E921196FA01A193B0839F91BE
:100FE0008F910895222369F7EACF7AE0979F902D99
:100FF000879F802D910D1124089580919A0381304F
:1010000019F482E080939A0380919A03833019F453
:1010100084E080939A030895E3E0F0E089E0809310
:101020005700849190E08670863009F491E0892F12
:1010300008951F93182F0E940C08882379F09FB7FA
:1010400081E08093A105F894A89588E180936000E1
:1010500010936000112309F0A8959FBF1F91089578
:10106000382F20E080913305909134058227932713
:1010700040E061E270E19C01220F331F97FF04C042
:10108000C9018627972701C0C9014F5F483099F7EA
:101090009093340580933305089587E38093D003BC
:1010A00080E092ECA1E0B0E08093D1039093D20372
:1010B000A093D303B093D40387E08093DD0380EC47
:1010C0009AECA9E8B6E38093D5039093D603A09356
:1010D000D703B093D80385E08093DE038DEE9EEFB7
:1010E000ADEABEED8093D9039093DA03A093DB03BE
:1010F000B093DC03AFEDB3E080E090E0863010F019
:10110000E0E004C0FC01EF57FC4FE081ED93019655
:101110008831910599F782E08093F7038AE0809304
:10112000F803089580EC97EFAAEBB7E380939D0353
:1011300090939E03A0939F03B093A00380E090E060
:10114000A0E0B0E58093A1039093A203A093A30332
:10115000B093A403E5EAF3E080E081938F5F8031F0
:10116000E1F708958436910520F4BC0180E090E019
:1011700025C08E3B910550F48A559040BC0180E01B
:1011800090E02AE030E040E050E016C0823D91055A
:1011900050F4845B9040BC0180E090E024E630E0B5
:1011A00040E050E009C08D5C9040BC0180E090E0E0
:1011B00028E532E040E050E00E94892F24E630E04C
:1011C00040E050E00E94892F089590E08C599F4F95
:1011D0000E94B2080895DC019896EC91F0E0E77067
:1011E000F070E758FC4F808108958F929F92AF92E4
:1011F000BF92CF92DF92EF92FF920F931F938C01D9
:101200000E94EB08D80197962C9130E043E150E022
:10121000249FF001259FF00D349FF00D1124EB5415
:10122000FD4F80809180A280B38090E00F96AA2726
:1012300097FDA095BA2FBC01CD0120E43FE14DE719
:1012400050E00E94892FA50194010E94BB2F6901E3
:101250007A0180ED97E0A0E0B0E0C80ED91EEA1E4A
:10126000FB1ED80198968C91887181F060E07EEE2B
:101270008AEB9BE0A50194010E94BB2F28513C4FB3
:101280004F4F5F4FC20ED31EE41EF51E87EE93E054
:10129000A0E0B0E0C80ED91EEA1EFB1EC701B601D1
:1012A00028EE33E040E050E00E94BB2FCA01B901B4
:1012B00028EE33E040E050E00E94892F1F910F910B
:1012C000FF90EF90DF90CF90BF90AF909F908F9066
:1012D00008958F3F910509F010F480E0089522E011
:1012E0008030920710F481E008958050934010F010
:1012F00083E0089582E00895CF92DF92FF920F93EA
:101300001F93CF93DF93F82FEB016A01182F1695E7
:10131000E0E088819981D6018C938A819B81119626
:101320008C9311978C819D8112968C9312978E814C
:101330009F8113968C931397288139814A815B8111
:101340006C817D818E819F819295990F990F907C00
:10135000832F8370982B852F8370880F880F982B8D
:10136000872F83708295807F982B14969C9385E0BD
:1013700090E0C80ED91E2896EF5F1E1750F6F0FFBA
:1013800021C0888199810E946909F82E8A819B81F8
:101390000E946909182F8C819D810E946909082F7C
:1013A0008E819F810E946909F294FF0CFF0C70EC02
:1013B000F7221295107F1F29182B000F000F012B09
:1013C000D6010C93DF91CF911F910F91FF90DF9089
:1013D000CF90089523E08032920718F420E030E0A7
:1013E00026C023E0883E920748F49C012F513340E9
:1013F00054E0369527955A95E1F719C027E0803DCE
:10140000920720F49C012C5D334011C028E08839FC
:10141000920718F02FEF33E00AC09C01285C374098
:1014200044E0369527954A95E1F72D503C4FC90188
:1014300008958C30910548F49C0174E0220F331F0D
:101440007A95E1F7285D3C4F17C023E0843F92076F
:1014500020F49C0124523C4F0FC024E080309207BE
:1014600018F020E938E008C09C012657334F64E0AB
:10147000220F331F6A95E1F7C90108959C01369543
:10148000279525753575821B930B9C0136952795FD
:10149000369527952373337383739373280F391FFE
:1014A000C901E4E096958795EA95E1F7820F931FCD
:1014B0008F709F7021E031E0AC01429FC001439FDB
:1014C000900D529F900D1124892F0895882339F093
:1014D00042980000419A0000429A00000895429804
:1014E000000041980000429A00000895429A0000CE
:1014F00086B142980000817008950F931F93082FC2
:101500005C9A42985C9810E0802F80780E94660A6E
:10151000000F1F5F1830C1F742981F910F91089577
:101520008F770E947D0A08950F931F93082F10E074
:10153000802F80780E94660A000F1F5F1830C1F765
:1015400042981F910F9108950F931F93429880E046
:1015500000E0182F110F0E94760A810F0F5F0830EC
:10156000C1F71F910F9108950E94900A0E94A40A4A
:101570005C9A08951F93162F80680E947D0A812F20
:101580000E94940A5C9A1F9108951F931091D903A9
:101590001827E0EDF3E0E80FF11D89E767850E9469
:1015A000BA0A8DE3612F0E94BA0A82E4612F0E9479
:1015B000BA0A1F91089586E20E94B40A08950F9313
:1015C0001F938C018CE1F80164810E94BA0A8DE1BD
:1015D000F80165810E94BA0A8EE1F80166810E94D5
:1015E000BA0A80E2F80167810E94BA0A81E2F80132
:1015F00060850E94BA0A82E2F80161850E94BA0AF7
:1016000083E2F80162850E94BA0A84E2F8016385E8
:101610000E94BA0A85E2F80164850E94BA0A8AE249
:10162000F80165850E94BA0A8EE6F80166850E9477
:10163000BA0A8FE6F80167850E94BA0A80E7F801C6
:1016400060890E94BA0A81E7F80161890E94BA0A9A
:1016500082E7F80162890E94BA0A1F910F910895EA
:10166000EF92FF920F931F93CF93DF937B018C0137
:10167000603028E372072CE982072CE1920728F5F5
:1016800020E836E948E950E00E94BB2FE90168975D
:10169000B90180E090E020E839E647E65FEF0E947C
:1016A000892F6E0D7F1D801F911F22E0660F771F0F
:1016B000881F991F2A95D1F721E732E040E050E0DA
:1016C0000E94BB2F890180E421C020E03DE241E37C
:1016D00051E00E94BB2FE9016897B90180E090E0DA
:1016E00020E033ED4EEC5EEF0E94892F6E0D7F1DE2
:1016F000801F911F660F771F881F991F21E732E017
:1017000040E050E00E94BB2F890180E69E012F71CE
:10171000622F680F85E70E94BA0A86E7612F0E9450
:10172000BA0A87E7602F0E94BA0ACDB7DEB7E6E0B3
:101730000C9420309F92AF92BF92CF92DF920F9382
:10174000DF93CF9300D000D0CDB7DEB7982E83E0E3
:101750000E94B40A8093F90384E00E94B40A809343
:10176000FA0386E060E00E94BA0A87E061E00E9426
:10177000BA0A89E06FE70E94BA0A8AE065E00E942F
:10178000BA0A8BE062E10E94BA0A8CE065E10E942D
:10179000BA0A8DE06DEF0E94BA0A8EE060E00E9406
:1017A000BA0A992019F084E193E008C08091F70308
:1017B00023E1829FC00111248B549D4F0E94DF0AB8
:1017C00080E36CE80E94BA0A82E36FE00E94BA0AE2
:1017D00083E362E40E94BA0A84E36AE00E94BA0AE0
:1017E00085E36AE20E94BA0A86E36DE20E94BA0AC1
:1017F00087E364ED0E94BA0A88E360E00E94BA0AB7
:1018000089E360E00E94BA0A992049F055E8A52EC4
:1018100051ECB52E51ECC52E5EEDD52E08C0A09032
:10182000D903B090DA03C090DB03D090DC030AE365
:101830008D2D9927AA27BB2789839A83AB83BC83E5
:10184000802F69810E94BA0A802F8B5F69810E9474
:10185000BA0ADC2CCB2CBA2CAA240F5F0E3341F72A
:1018600083E46FEF0E94BA0A84E46FEF0E94BA0A21
:1018700085E46FEF0E94BA0A86E46FEF0E94BA0A0D
:10188000992019F08DE666E003C08DE66091DD03D6
:101890000E94BA0A89E760E00E94BA0A8AE760916A
:1018A000DE030E94BA0A83E760E00E94BA0A84E776
:1018B00060E00E94BA0A992029F060EC7AEC89E88D
:1018C00096E308C06091D5037091D6038091D70349
:1018D0009091D8030E94300B0F900F900F900F90B3
:1018E000CF91DF910F91DF90CF90BF90AF909F90FD
:1018F000089587E061E00E94BA0A8EE764E20E94E0
:10190000BA0A88E063E00E94BA0A88E060E00E94B8
:10191000BA0A87E065E00E94BA0A85E062E00E94A8
:10192000BA0A83E00E94B40A8093F90384E00E941B
:10193000B40A8093FA030895582F40919E04842F8F
:1019400090E0FC01EF70F0709F012F5F3F4F64E06B
:10195000959587956A95E1F72817390751F0E25771
:10196000FB4F5083842F8F5F8F70407F842B809339
:101970009E0408951F920F920FB60F9211241F9389
:101980002F933F934F935F936F937F938F939F9387
:10199000AF93BF93CF93DF93EF93FF93C0918600F4
:1019A000D09187002091E0043091E1048091BF0440
:1019B000882309F062C0BE01621B730B2091A10352
:1019C0003091A2034091A3035091A40325FD02C0CE
:1019D0007695679589E0653C7807B8F18091470373
:1019E000BCE15695479537952795BA95D1F72115BE
:1019F00031054105510521F421E030E040E050E09F
:101A000090E0A0E0B0E0281739074A075B07D0F460
:101A1000809147038F3FB1F020E00EC0E22FF0E04D
:101A2000EE0FFF1FDF01A054BB4F8D919C91E95D2C
:101A3000FC4F918380832F5F80914703281770F3B9
:101A40001092BE041092470318C082E06D3B7807E5
:101A500060F180914703803140F510914703CB013D
:101A60000E94EA09E12FF0E0EE0FFF1FE054FB4F68
:101A7000918380831F5F10934703D093E104C09349
:101A8000E004FF91EF91DF91CF91BF91AF919F91D2
:101A90008F917F916F915F914F913F912F911F9106
:101AA0000F900FBE0F901F9018958FEF80934703F4
:101AB000E4CF83E0809380008AE980938100809165
:101AC000A10386FD05C08091810080648093810020
:101AD0008FEF9FEF909389008093880080916F0033
:101AE000806280936F0008956F3018F0869580585B
:101AF000089589E0689F802D11240895882319F4A2
:101B000060E071E002C063E071E087E396E00E946C
:101B10003D2D0895A0E0B0E0E0E9FDE00C94023036
:101B2000182F0E94EE299B01AC0180912D05909108
:101B30002E05A0912F05B091300569017A01C81AD0
:101B4000D90AEA0AFB0AD701C60189589341A04085
:101B5000B04010F010922C0520932D0530932E05E7
:101B600040932F05509330052091BF04822F815060
:101B70008230E8F580912C05882309F44FC181302B
:101B800011F482E0BCC1803108F035C1E82FF0E0EB
:101B9000E054FB4F10838F5F80932C05803109F058
:101BA000B0C1A2ECB4E0213039F41196EC91119758
:101BB000E695E6958C9109C08D919C911197E92F3E
:101BC000E695E695E69596958795E03140F4F0E048
:101BD00090E0EE0FFF1FE95DFC4F91838083109230
:101BE000BE04129684E0A03DB807E9F68AC123300E
:101BF00009F004C180912C05882321F41F3009F0DD
:101C000080C10CC1883130F4E82FF0E0E154FB4F83
:101C1000108374C1883109F0EEC0112309F0EBC0C4
:101C2000C0E0D0E00BE010E0DE0163E0AA0FBB1FD4
:101C30006A95E1F7C09FB001C19F700DD09F700DF4
:101C40001124FB01E054FB4F80812181922F97707A
:101C500095958795FD01EE0FFF1FE95DFC4F918380
:101C60008083FB01EF53FB4F3081369536953695D7
:101C70002181422F4295440F407E842F832B26954D
:101C800026952695922F977095958795FD01EE0FD5
:101C9000FF1FE75DFC4F91838083FB01EE53FB4FF9
:101CA000808182958695869583704181942F990FC6
:101CB000990F292F282B429546954695437082818E
:101CC0008170880F880F382F342B35952795FD01AB
:101CD000EE0FFF1FE55DFC4F31832083FB01EC53CA
:101CE000FB4F308136952181422F479544274795F8
:101CF000842F832B2695922F977095958795FD01BC
:101D0000EE0FFF1FE35DFC4F91838083FB01EB53DC
:101D1000FB4F308132953F702181422F4295407FA9
:101D2000842F832B22952F70922F977095958795EE
:101D3000FD01EE0FFF1FE15DFC4F91838083FB01EE
:101D4000EA53FB4F8081881F8827881F4181942F89
:101D5000990F292F282B441F4427441F8281837009
:101D6000880F382F342B35952795FD01EE0FFF1F77
:101D7000EF5CFC4F31832083FB01E853FB4F308144
:101D8000369536952181422F4295440F440F407C71
:101D9000842F832B26952695922F9770959587955E
:101DA000AA0FBB1FFD01ED5CFC4F9183808367533D
:101DB0007B4FFB0120812295269527704181342F8E
:101DC000330F330F330F832F822B942F92959695D9
:101DD000977095958795AB5CBC4F11969C938E93AD
:101DE0002196C230D10509F01FCF8091D60483FD22
:101DF00002C01092BE0410922C0583C0243009F05A
:101E000080C040912C05442359F4183AB1F4109243
:101E100034051092330588EA0E94300881E06FC0D3
:101E2000413019F41093310504C0423031F410935D
:101E30003205812F0E9430085DC060913205262F47
:101E400030E0220F331FE42FF0E0C90102968E1715
:101E50009F0734F0433268F7E354FB4F1083E9CF18
:101E60002D5F3F4F4091330550913405E217F30742
:101E700049F4912F80E04827592750933405409327
:101E8000330538C0812F90E04817590789F58091B4
:101E90003105813069F5613118F080E180933205B8
:101EA000D090320540ECE42E44E0F42E00E010E047
:101EB0001BC0F701D081C0E0818190E08C2B9D2B6D
:101EC00033E0969587953A95E1F70E94EA09F80183
:101ED000EE0FFF1FE95DFC4F918380830F5F1F4F63
:101EE00082E090E0E80EF91E0D1518F31092BE0482
:101EF00010922C0580912C05882319F08F5F809318
:101F00002C05CDB7DEB7E8E00C941E30FF920F939E
:101F10001F93CF93DF93182F092FF62E8EE30E9485
:101F2000BA0A212F302FC901EC0110E005C08FE75C
:101F300069910E94BA0A1F5F1F15C8F385E064E02B
:101F40000E94BA0A83E00E94B40A8093F90384E0F5
:101F50000E94B40A8093FA030E94EE296093FB0367
:101F60007093FC038093FD039093FE0387E069E088
:101F70000E94BA0A81E080939A03CDB7DEB7E5E00C
:101F80000C9421300E94860F80919A038130D9F4FD
:101F90000E94EE292091FB033091FC034091FD0348
:101FA0005091FE03621B730B840B950B605A7648AD
:101FB0008140904040F4E8CF87E396E067E071E02D
:101FC0000E943D2D089580919A038130A9F30895D0
:101FD00087E396E06EE70E94F52E0895A0E0B0E05A
:101FE000E4EFFFE00C9401306C0187E396E06EE7CC
:101FF0000E94F52E760100E010E0C0E0D0E0B0E2F3
:10200000BB2E0AC00830110521F49E012095F6016F
:1020100020870894E11CF11CF7016081862F8D5701
:10202000823040F487E396E06DE70E94F52EF701D9
:1020300060816B2587E396E00E94F52E011511055E
:1020400051F0F70180819E01280F311DC32FDD273C
:10205000C20FD31FD0700F5F1F4F0930110591F6CB
:10206000CDB7DEB7E9E00C941D30A9E0B0E0EBE3BA
:10207000F0E10C940830382FE62F8091A30490E013
:10208000019664E270E00E94A82F982F8093A30429
:1020900088E9898380E18A83913071F0913028F05A
:1020A000923099F09330E1F416C085E08B8381EF94
:1020B0008C832F5F2D8317C09B8381EF8C8384E6F5
:1020C000489FC00111249D830EC084E08B8381EF63
:1020D0008C833D8308C09B8381EF8C83ED8303C099
:1020E0000E94E80F04C0CE0101960E94EE0F2996CF
:1020F000E2E00C9424300F931F93CF93DF93182FBB
:10210000092F87E396E06EE70E94F52E212F302FEE
:10211000C901EC0110E000E288818D57823040F463
:1021200087E396E06DE70E94F52E888180278883FB
:1021300087E396E069910E94F52E1F5F193061F7E1
:1021400087E396E06EE70E94F52EDF91CF911F9115
:102150000F910895A9E0B0E0E0EBF0E10C940830B5
:10216000382F8091A304882379F48EEF89833A83F2
:102170006B83842F90E0959587958C832D831986AA
:1021800018861F821E822FC040919E04842F90E0EB
:102190009C012F70307054E0959587955A95E1F722
:1021A0008217930721F18DEF89831A821B82DE014A
:1021B000149620E008C0E257FB4F80818D93405F6A
:1021C0002F5F263069F0842F90E0FC0134E0F59514
:1021D000E7953A95E1F78F709070E817F90759F78E
:1021E00040939E042A83CE0101960E947B10809129
:1021F000A30490E0019666E070E00E94A82F80930F
:10220000A3042996E2E00C9424309F92AF92BF92EF
:10221000CF92DF92EF92FF920F931F93B82EA62ECC
:10222000D42EC22E902E0E94EE297B018C0180912B
:102230008D0420919F043091A0044091A1045091FD
:10224000A2048823B1F0D801C701821B930BA40B11
:10225000B50B815E9E42A040B04020F12C2DDC14D5
:1022600008F42D2D8B2D6A2D422F292D0E9435101B
:1022700011C0D801C701821B930BA40BB50B81536E
:102280009547A040B04070F08B2D6A2D4D2D2C2D20
:102290000E94AA10E0929F04F092A0040093A1046F
:1022A0001093A2041F910F91FF90EF90DF90CF90B9
:1022B000BF90AF909F90089587E396E060910004EF
:1022C0000E94F52E08951F93182F87E396E0612F43
:1022D0000E94F52E809100048127809300041F91B5
:1022E00008951F93192F0E946311812F0E9463117B
:1022F0001F910895DF92EF92FF920F931F93D82EB4
:102300007B011092000407E316E0C80165EB0E9410
:10231000F52EC80162E60E94F52E8D2D0E946311F4
:10232000C7010E9471111F910F91FF90EF90DF90F4
:102330000895E82FF0E0E456FC4FE185E03158F4D1
:10234000F894F0E0EE0FFF1FE95DFC4F0190F08183
:10235000E02D78940DC0E03129F0E13129F0E0E082
:10236000F2E006C082E101C083E10E94422BFC0141
:10237000CF0108958EE060E00E94732A8FE061E053
:102380000E94732A80E161E00E94732A82E060E08B
:102390000E94732A84E061E00E94732A0895CF931B
:1023A000DF93EC01009741F186E061E00E94DF2AB3
:1023B0009E0140E050E068E478EE81E090E00E9409
:1023C000DD2FC901DA018F3F9105A105B10531F07B
:1023D00028F08FEF90E0A0E0B0E008C00097A105E2
:1023E000B10521F481E090E0A0E0B0E08093B3007B
:1023F0008091B000806107C086E060E00E94DF2A23
:102400008091B0008F7E8093B000DF91CF910895CE
:10241000A0E2B0E0EEE0F2E10C9400308CE00E942B
:10242000B40A882389F587E396E063E171E00E94AE
:102430003D2D439A299A80E00E949A0B0E94790CC4
:102440004398299821C087E396E00E94BC2E482F2C
:102450008091BF04882321F0842F0E948A0D14C02C
:1024600080912A05E82FF0E031969F012F7130709E
:1024700031978091290590E02817390729F0E0501D
:10248000FB4F408320932A0587E396E00E94822E2B
:10249000892BC9F680919A03843009F08EC00E947E
:1024A000EE296093AE047093AF048093B0049093D0
:1024B000B104611571058105910561F481E090E039
:1024C000A0E0B0E08093AE049093AF04A093B0047A
:1024D000B093B1048091BA049091BB048160909351
:1024E000BB048093BA0483E080939A038FE70E9431
:1024F000900A07EF14E00E94A40AF80181938F016B
:10250000F5E000301F07B9F74091E2048091F7042D
:10251000282F30E0842F90E08227932786FF40C049
:1025200080E448274093E204C90188739070C897FB
:1025300009F510E014C01F5F8091F803E12FF0E06F
:1025400084FF06C0E950FB4F80810E949C0C07C0AD
:10255000E950FB4F87E396E060810E94F52E212F22
:1025600030E08091F70490E08770907082179307B5
:1025700014F716C02F733070232B91F48091F80458
:102580008093B2048091F9048093B4048091FA049A
:102590008093B5048091FD048093BC041092BD0427
:1025A00080912B05813019F482E080932B05809176
:1025B0002B05833011F410922B050E94EE295B014C
:1025C0006C018091B6049091B704A091B804B091C9
:1025D000B9040097A105B105C9F086017501E81A93
:1025E000F90A0A0B1B0BD801C701885B9B40A0406E
:1025F000B04060F00E94DB0A8093B3041092B604EE
:102600001092B7041092B8041092B90480ED93E0D0
:102610000E94F5082091AA043091AB044091AC04CB
:102620005091AD0486017501E21AF30A040B150BF3
:10263000E616F7060807190708F411C1A092AA04C4
:10264000B092AB04C092AC04D092AD04A895809136
:10265000BE048830A0F08091A1039091A203A091C4
:10266000A303B091A403FCE1B695A7959795879530
:10267000FA95D1F70097A105B10509F091C18091B4
:10268000BE048F5F8093BE04E090AE04F090AF0470
:102690000091B0041091B104E114F1040105110599
:1026A00011F180ED93E00E94F508AE18BF08C00A52
:1026B000D10A6A157B058C059D0588F48091A103DC
:1026C00084FD04C080ED97E00E94CF111092AE040B
:1026D0001092AF041092B0041092B10404C080E0D4
:1026E00090E00E94CF119091E204907C9093E204DC
:1026F00000912A05109129050117B1F180912B0550
:10270000823091F590589093E20480ED93E00E941E
:10271000EB08893010F048E002C0482F415030E00B
:1027200013C03F5FA32FB0E0812F90E0FC01E05089
:10273000FB4F2081FD01EE51FB4F2083A05EBA4F7D
:102740002C930196182F1F71341710F4101749F7A6
:1027500010932905832F895C9091E204892B809343
:10276000E204309320051AC020912B052430D1F4C7
:1027700090912005E1E2F5E0A3EEB4E0292F30E0EE
:102780002E0F3F1F02C081918D93E217F307D9F7F7
:10279000995C8091E204982B9093E20483E080930B
:1027A0002B0538C08091A504823061F4916090932C
:1027B000E204439A299A05EA13E07E010894E11C99
:1027C000F11C11C09093E20443982998222319F434
:1027D00081E080932B0580912B05833061F784E0A5
:1027E00080932B05E8CFF80181918F010E94991108
:1027F000F701819391937F01F3E0053B1F0799F760
:102800008091F8038770BE016F5F7F4F43EE54E005
:102810000E947C0985B1846285B98091A4040E94DC
:10282000C50A80ED93E00E94EB08682F82EE94E0E9
:102830000E94860FE091A404EF5FE093A404E831C6
:1028400031F0F0E0E053FC4F8785882341F410928B
:10285000A40405C0439A299A89E08093BE0480911C
:10286000F803887171F180919A03823051F580915B
:10287000BA049091BB04880F991F9093BB04809376
:10288000BA0483E080939A030E94790C0E94EE2997
:102890006093B6047093B7048093B8049093B9041E
:1028A000611571058105910561F481E090E0A0E07A
:1028B000B0E08093B6049093B704A093B804B093AB
:1028C000B9048091F80384FF1EC08091BA049091EE
:1028D000BB048E7F0E943E0A182F8091B204609143
:1028E000BC040E94740D082F8091B304612F0E94D4
:1028F000740D282F8091B4046091B504402F00918D
:102900009B030E94051185B18B7D85B98091A5043B
:102910008130D1F0813020F0823009F047C034C0DE
:1029200087E00E94122B892B09F040C081E0809340
:10293000A5040E94E0296093A6047093A7048093E5
:10294000A8049093A90432C087E00E94122B892B1F
:1029500021F50E94E0292091A6043091A70440911E
:10296000A8045091A904621B730B840B950B695E3C
:10297000734080409040D0F082E08093A50480EDC9
:1029800097E00E94CF1112C087E00E94122B892B82
:1029900069F080E090E00E94CF111092A50406C07B
:1029A0008091BE04883009F057CF54CFA096EAE05A
:1029B0000C941C3086E061E00E94732A86E060E09F
:1029C0000E94DF2A82E08093B00085E08093B1000E
:1029D00083E061E00E94732A83E060E00E94DF2AC6
:1029E00008951F93182F0E94EE2960939F047093FF
:1029F000A0048093A1049093A20410938D0411234A
:102A000029F440E855E260E070E004C040E051EE97
:102A100060E070E087E396E00E94FB2D1F9108952F
:102A2000ACE1B0E0E6E1F5E10C9400300E94EE2963
:102A30007B018C0181E00E949A0B84E7A82E6E0135
:102A40000894C11CD11CB3E0BB2EA982C60161E071
:102A50000E94C20FB0929A030E94790C6AEF70E054
:102A600080E090E00E94142A80919A03833009F05C
:102A70007DC087E396E00E94822E892B09F076C004
:102A80000E94EE296E197F09800B910B6058734CE0
:102A9000894C914008F06AC0D8CF8FE70E94900A15
:102AA0000E94A40A843509F05CC089830E94A40AAC
:102AB000182F00E010938C0400938B040E94A40A4A
:102AC000080F111D10938C0400938B040E94A40A1C
:102AD00080938A040E94A40A80938904813108F0BB
:102AE00040C0FF2407C00E94A40A07591B4FF801E9
:102AF0008083F3940F2D10E08091890490E0880F7B
:102B0000991F0817190778F380E78983CE0101968A
:102B100061E00E94C20F83E080939A030E94790CC7
:102B200062E370E080E090E00E94142A80919A03B2
:102B30008330A9F08FE70E94900A0E94A40A803592
:102B400081F4898305EB13E00E94A40AF8018193C4
:102B50008F01F3E0003D1F07B9F781E003C082E079
:102B600001C083E06C96EAE00C941C3080919A03DB
:102B7000833009F092CFF3CF83E00E94B40A8093B0
:102B8000F90384E00E94B40A8093FA0387E061E0CD
:102B90000E94BA0A6AE070E080E090E00E94142A85
:102BA0000E94790C000008950F931F93082F19C0FD
:102BB000439A299A64E670E080E090E00E94142A2B
:102BC0004398299864E670E080E090E00E94142A1F
:102BD0001F5F101768F36CE271E080E090E00E94E4
:102BE000142A10E0F6CF482F392F25E00DC0F999AF
:102BF000FECF1FBA842F932F92BD81BD60BD0FB64B
:102C0000F894FA9AF99A0FBE215059F0F999FECF2B
:102C1000842F932F92BD81BDF89A80B5681739F73C
:102C2000089582E00E94D4150895A0E0B0E0EBE1A1
:102C3000F6E10C94F92F482E562EEE24FF2488241A
:102C40009924C0E0D0E0CC24DD2476E4372E04C003
:102C500055245394CC24DD24442069F480919B03B3
:102C6000839DE00111246CE9E62E63E0F62E59E124
:102C7000852E912C1DC021E0421671F480919B039A
:102C8000839DE00111246B9640EDE42E43E0F42E89
:102C900039E2832E912C0CC032E0431649F42BE923
:102CA000E22E23E0F22E91E0892E912CC8E1D1E0B2
:102CB0003E016C0C7D1C1092340510923305E3012B
:102CC0001BC0552059F4F999FECFD2BDC1BDF89A69
:102CD00080B5F701E00FF11F808307C0F701E00F17
:102CE000F11FCE0160810E94F3150E0D1F1DF8012A
:102CF00080810E94300821969E012619022F10E043
:102D000008151905F0F2CE015520D9F4F999FECF36
:102D1000D2BDC1BDF89A20B5F999FECF2196D2BD9A
:102D2000C1BD2197F89A80B590E0B22EAA248A29D5
:102D30009B2920913305309134052817390759F420
:102D400087CF2196609134050E94F315CE016091E2
:102D500033050E94F31580E291E0C80ED91E91EE72
:102D6000C91692E0D90608F477CF852DCDB7DEB726
:102D7000E1E10C94153080E061E00E94151681E0DD
:102D800061E00E941516089580E060E00E9415162B
:102D9000882331F081E060E00E941516882331F429
:102DA0000E9492080E944D080E94BB16089582E07E
:102DB00061E00E941516089582E060E00E941516F9
:102DC00080919B03843020F010929B030E94D716C1
:102DD00008951F93182F0E94DC1680919B03811782
:102DE00031F0143020F410939B030E94D7161F91EA
:102DF00008951092670485E6E2E0F4E0DF011D9299
:102E00008A95E9F708951F93182F8F3711F08830AE
:102E1000E1F5E0916704EE2309F455C0E150E09339
:102E20006704F0E0EE5FFB4F108287E396E06DE011
:102E30000E94F52E10E00AC0E12FF0E0EE5FFB4F9C
:102E400087E396E060810E94F52E1F5F8091670402
:102E5000181790F387E396E060E20E94F52E87E36F
:102E600096E06DE00E94F52E10E00AC0E12FF0E040
:102E7000EE5FFB4F87E396E060810E94F52E1F5FB7
:102E800080916704181790F31CC08B3119F40E94CD
:102E9000F9161FC08D30E9F08A30D9F080916704AF
:102EA000843688F487E396E0612F0E94F52E8091A6
:102EB0006704E82FF0E0EE5FFB4F10838F5F809395
:102EC000670480E007C087E396E067E00E94A92BD3
:102ED000F8CF81E01F9108951F93CF93DF93CFED3B
:102EE000D3E010E03BC087E396E062E271E00E942D
:102EF0003A2D87E396E0612F4AE050E00E94B72C1C
:102F000087E396E06FE271E00E943A2D699170E0EC
:102F100080E090E02091DE0330E040E050E00E944D
:102F2000892F20E137E240E050E00E94892FDC0148
:102F3000CB014091D5035091D6036091D703709196
:102F4000D803480F591F6A1F7B1F87E396E02AE0CA
:102F500030E00E947E2C1F5F183119F08881882391
:102F600011F6DF91CF911F910895EF92FF920F9389
:102F70001F93882339F487E396E061E77AE00E94A3
:102F8000C72B3BC090E00E94B20824E630E040E04E
:102F900050E00E94BB2F122F032FF42EE52E622F3C
:102FA000732F842F952F2AE030E040E050E00E94FC
:102FB000BB2F87E396E0BA01A9012AE030E00E9426
:102FC0006F2C87E396E06EE20E94A92B612F702F91
:102FD0008F2D9E2D2AE030E040E050E00E94BB2F74
:102FE000AB01BC0187E396E02AE030E00E946F2C41
:102FF00087E396E063E70E94DB2B1F910F91FF9020
:10300000EF900895FF920F931F93CF93DF9387E381
:1030100096E067E67AE00E94882B8091B5038130C4
:1030200041F487E396E06EE47AE00E94C72BFF2428
:103030006DC0823029F487E396E067E37AE0F5CF4C
:10304000843029F487E396E063E27AE0EECF8530BE
:1030500071F787E396E068E17AE0E7CFCF2DD0E023
:10306000C930D1051CF06F2D685C02C06F2D6F5CFC
:1030700087E396E00E94A92B87E396E060E17AE07F
:103080000E94882BBE016F5F7F4F87E396E04AE086
:1030900050E00E94132D87E396E065E07AE00E94FD
:1030A000882B8E010B541C4FD8011196EC91E03205
:1030B000F8F487E396E068EF79E00E94882BF80146
:1030C0008181803130F087E396E063E371E00E9414
:1030D0003A2DCB54DC4F698170E06F7070706F5F78
:1030E0007F4F87E396E04AE050E00E94262D0DC016
:1030F000F0E0EF70F070EE0FFF1FE75BFC4F6081B8
:10310000718187E396E00E943D2DF39480918A04BB
:10311000F81608F4A3CF87E396E06DED79E00E94FE
:10312000882B8091CD030E94B51787E396E062EC6F
:1031300079E00E94882B8091CE030E94B51787E327
:1031400096E067EA79E00E94882B8091CF030E9485
:10315000B51787E396E06CE879E00E94882B4091F0
:10316000C5035091C6036091C7037091C803411510
:1031700051056105710539F187E396E02AE030E0F9
:103180000E947E2C87E396E069E579E00E94882B17
:103190008091C9030E94E508AB01BC0187E396E07A
:1031A0002AE030E00E947E2C87E396E065E379E038
:1031B0000E94882B87E396E06091CA034AE050E0C2
:1031C0000E94C92C06C087E396E06CE279E00E9479
:1031D000C72B87E396E06FE079E00E94882B60912F
:1031E000CB037091CC0387E396E04AE050E00E9465
:1031F000A32C87E396E062EF78E00E94882B609131
:10320000C403603450F470E06F5F7F4F87E396E053
:103210004AE050E00E94262D06C087E396E069EE62
:1032200078E00E94C72B87E396E06CEC78E00E9480
:10323000882B8091C30380FD03C065E371E002C069
:1032400069E371E087E396E00E943D2D87E396E015
:103250006FEA78E00E94882B8091C30382700E94FD
:103260007E0D87E396E060E978E00E94882B8091EC
:10327000C30384700E947E0D87E396E061E778E0E7
:103280000E94882B8091C30388700E947E0DCDB769
:10329000DEB7E5E00C9421301F93CF93DF9387E3F3
:1032A00096E06BEB7BE00E94882B4091D503509118
:1032B000D6036091D7037091D80387E396E02AE0A4
:1032C00030E00E947E2C87E396E065EA7BE00E9476
:1032D000882B4091D9035091DA036091DB03709100
:1032E000DC0387E396E020E130E00E947E2C87E358
:1032F00096E06FE87BE00E94882B87E396E0609180
:10330000DD034AE050E00E94C92C87E396E069E7BC
:103310007BE00E94882B87E396E06091DE034AE021
:1033200050E00E94C92C87E396E063E67BE00E94B0
:10333000882BCFEDD3E010E012C0112331F087E3EA
:1033400096E06DE371E00E943A2D87E396E0699183
:103350004AE050E00E94B72C1F5F183119F08881B5
:10336000882359F787E396E00E94B12B87E396E024
:103370006DE47BE00E94882B87E396E06091F70381
:103380004AE050E00E94C92C87E396E068E37BE0C6
:103390000E94882BE091F803F0E0E770F070EE0FE8
:1033A000FF1FE759FC4F6081718187E396E00E941F
:1033B0003D2D87E396E063E27BE00E94882B8091BD
:1033C000F80390E0887190708830910589F0893019
:1033D00091051CF4892B39F01BC08031910569F0EF
:1033E0004897B1F40FC087E396E06AE17BE00EC036
:1033F00087E396E06EE07BE009C087E396E068E053
:103400007BE004C087E396E06EEF7AE00E94C72B72
:1034100087E396E06AEE7AE00E94882B4091D10320
:103420005091D2036091D3037091D40387E396E067
:103430002AE030E00E947E2C87E396E061ED7AE09E
:103440000E94882B8091A10380710E947E0D87E3EA
:1034500096E068EB7AE00E94882B8091A10380744B
:103460000E947E0D87E396E06FE97AE00E94882B48
:103470008091A10380720E947E0D87E396E062E84E
:103480007AE00E94882B80ED93E00E94F508AB0162
:10349000BC0187E396E02AE030E00E946F2C87E3CE
:1034A00096E06DE77AE00E94882B80ED93E00E9421
:1034B000F5089B01AC0160E472E48FE090E00E94AB
:1034C000BB2F87E396E0BA01A9012AE030E00E9411
:1034D0006F2C87E396E06AE77AE00E94C72BDF91C2
:1034E000CF911F910895EF92FF920F931F937C014C
:1034F00007E316E0C8016F2D70E04AE050E00E943B
:10350000922CC8016EE20E94A92BB70184E0769547
:1035100067958A95E1F76F707070C8014AE050E0D6
:103520000E94922CC8016EE20E94A92B8FE0E82233
:10353000FF24C801B7014AE050E00E94922C1F917D
:103540000F91FF90EF9008950F931F93CF93DF9308
:10355000209101042F3FA9F587E396E061EF75E024
:103560000E94882B81E793E00E94731A87E396E01C
:1035700060ED75E00E94882B80918B0490918C0403
:103580000E94731A87E396E06DE975E00E94C72BED
:1035900087E396E06AE775E00E94C72B87E396E031
:1035A00062E675E00E94C72B87E396E06DE375E065
:1035B0000E94C72B87E396E00E94B12B0E9402185D
:1035C00069C012160CF066C0332727FD3095809134
:1035D0008A0490E0821793070CF45CC087E396E0BE
:1035E00068E275E00E94882B60910104772767FDEF
:1035F000709587E396E04AE050E00E94262D87E32D
:1036000096E06DEF74E00E94882B08E210E03AC06B
:10361000C12FD0E0CC0FDD1FC759DB4F288130E030
:1036200080910104992787FD909501972817390704
:1036300041F587E396E06FE371E00E943A2D87E35E
:1036400096E0602F4AE050E00E94B72C87E396E0B6
:1036500063E471E00E943A2DE981F0E0EF70F070D0
:10366000EE0FFF1FE75BFC4F6081718187E396E0FF
:103670000E943A2D87E396E067E471E00E943A2DBC
:103680000F5F1F5F80918904181710F287E396E09F
:103690000E94B12BDF91CF911F910F910895ACE162
:1036A000B0E0E5E5FBE10C940230282F80910104A5
:1036B0008F3F09F042C1822F90E0FC013A97EF362C
:1036C000F10508F033C1EC5CFF4F0C942F3087E319
:1036D00096E069E471E0AEC087E396E069E471E0EA
:1036E0000E943D2D1CC187E396E065E571E00E94D4
:1036F0003D2D85E78983DE011296E5EBF3E08BE152
:1037000001900D928150E1F7CE0101966CE10E948B
:10371000C20F0E94790C83E080939A0368EC70E0FA
:1037200080E090E00E94142A80919A03843009F08E
:10373000FDC08FE70E94900A0E94A40A8983853504
:1037400009F0F4C087E396E06FED74E00E94C72BA8
:1037500087E396E061EC74E00E94C72B87E396E074
:1037600063EA74E0ACC087E396E06DE671E00E9426
:103770003D2D89E68983CE01019661E00E94C20F4A
:103780000E94790C83E080939A0368EC70E080E0FB
:1037900090E00E94142A80919A03843009F0C6C0F8
:1037A0008FE70E94900A0E94A40A89838E010E5F0F
:1037B0001F4FBDE1EB2EF12CEC0EFD1E0E94A40A62
:1037C000D8018D938D01AE15BF05C1F7A5EBB3E010
:1037D000FE0132968BE101900D928150E1F78981D3
:1037E000893409F0A3C087E396E065E874E00E949D
:1037F000C72B87E396E067E674E00E94C72B87E358
:1038000096E069E474E05BC087E396E067E871E006
:103810000E943D2D8EEF8093010488C020522750D6
:10382000922F905380918A04891738F487E396E0A9
:1038300066E971E00E943D2D79C0909301046FC04C
:1038400084E18093010487E396E062E174E037C08D
:1038500085E18093010487E396E06BED73E02FC070
:1038600086E18093010487E396E064EA73E027C071
:1038700087E18093010487E396E06AE573E01FC067
:1038800088E18093010487E396E069E473E017C060
:1038900089E18093010487E396E065E373E00FC05C
:1038A0008AE18093010487E396E060E273E007C059
:1038B0008BE18093010487E396E068EF72E00E9459
:1038C000C72B34C087E396E06EED72E00E94C72BF1
:1038D0008091C30391E01DC087E396E068EC72E03D
:1038E0000E94C72B8091C30392E013C087E396E048
:1038F00063EB72E00E94C72B8091C30394E009C080
:1039000087E396E068E972E00E94C72B8091C303C9
:1039100098E089278093C3038FEF809301040E946E
:10392000A41A04C087E396E00E94BC2E87E396E0C9
:103930000E94822E892BB1F762C1822F0E94031749
:10394000882309F45CC180916704882321F48FEFF8
:10395000809301044CC182E094E060E070E040E0BC
:1039600050E00E94A2069B01AC0160910104862FE9
:10397000992787FD9095A92FB92FFC013197EB313D
:10398000F10508F024C1ED55FF4F0C942F30E62FC0
:10399000FF27E7FDF09580918A0490E08E179F073E
:1039A0000CF415C1DA01C9010197A109B109809789
:1039B000A105B10548F0A8E2FA2E00E010E06F0181
:1039C0000894C108D10825C0EB54FC4F822F8150C8
:1039D0008083E5C0612F70E0660F771F67597B4FCA
:1039E000FB01808190E08C159D0591F48F2D90E076
:1039F000A0E0B0E082179307A407B50741F4F601F1
:103A0000EB54FC4FDB0111968C91818301E0F39420
:103A10001F5F809189041817E8F2BFC02F3F31055E
:103A20004105510511F008F0D2C02093CD03B7C075
:103A30002F3F31054105510511F008F0C8C0209312
:103A4000CE03ADC02F3F31054105510511F008F0FF
:103A5000BEC02093CF03A3C0809102048062803750
:103A600019F583E094E060E070E040E050E00E94EF
:103A7000A2069B01AC01DC01CB010197A109B109B0
:103A80000897A105B10508F0B5C0CA01B90124ED38
:103A900030E340E050E00E94892F9B01AC012A5E98
:103AA0003C4A4A46554E24C0863611F583E094E0E0
:103AB00060E070E040E050E00E94A2069B01AC0193
:103AC000DC01CB010197A109B1090797A105B10557
:103AD00008F090C0CA01B90128EA31E640E050E0A0
:103AE0000E94892F9B01AC01245E3C434E46544EFC
:103AF000211531054105510561F0DA01C901805CEC
:103B00009D49A845B54381509A45A246B24008F068
:103B10005EC02093C5033093C6034093C703509300
:103B2000C8033DC02F3F31054105510511F008F094
:103B30004EC02093C90333C0DA01C9010197A1091E
:103B4000B1098F3F9105A105B10508F040C0209350
:103B5000CA0325C0DA01C901845C9940A040B04085
:103B60008D549D41A040B04030F43093CC0320935D
:103B7000CB0301E001C000E02115310541055105ED
:103B800011F48FEF07C0213431054105510528F4A8
:103B9000822F81508093C40302C00023C1F0809122
:103BA00068048823D1F48091D9039091DA03A0911D
:103BB000DB03B091DC030196A11DB11D8093D903F5
:103BC0009093DA03A093DB03B093DC0306C087E392
:103BD00096E068EA71E00E943D2D0E94F9168FEF91
:103BE0008093010487E396E06AE00E94DB2B0E9449
:103BF000A41A05C021E030E040E050E07ECF6C9692
:103C0000E8E00C941E3087E396E06CE472E00E94DA
:103C1000C72B87E396E064E372E00E94C72B87E33B
:103C200096E00E94822E892B31F087E396E00E9475
:103C3000BC2E0E944F1B0E941015823019F0833059
:103C400069F405C087E396E066E172E004C087E3AB
:103C500096E06FEF71E00E94C72B08958FEF80937D
:103C60000104109268040E94A41A0CC087E396E035
:103C70000E94822E892B31F087E396E00E94BC2EB1
:103C80000E944F1B809101048E3F81F7089580911F
:103C90000104992787FD9095A92FB92FFC01319632
:103CA000EB30F10508F074C0E254FF4F0C942F3054
:103CB00087E396E064E678E00E94C72B81E793E013
:103CC0000E94731A87E396E06CE478E00E94C72BA9
:103CD00087E396E067E278E00E94C72B87E396E0EF
:103CE0006DEF77E00E94C72B87E396E06CED77E0FD
:103CF0000E94C72B87E396E06FEA77E00E94C72B0C
:103D000087E396E069E877E00E94C72B87E396E0B7
:103D100065E677E00E94C72B87E396E06EE377E0E5
:103D20000E94C72B87E396E00E94B12B0E944C199A
:103D30002FC087E396E061E277E028C087E396E052
:103D40006CEF76E023C087E396E067EE76E01EC076
:103D500087E396E068EC76E019C087E396E064E8D4
:103D600076E014C087E396E06FE676E00FC087E365
:103D700096E06AE576E00E94C72B87E396E064E16F
:103D800076E004C087E396E06EEF75E00E94C72BF3
:103D90006AE070E080E090E00E94142A04C087E3AB
:103DA00096E00E94BC2E87E396E00E94822E892B2B
:103DB000B1F70895A2E2B0E0E0EEFEE10C94F82F36
:103DC0008E010F5F1F4F80E1D8011D928A95E9F7A0
:103DD00087E396E066EC71E00E943D2D0E94BC15E1
:103DE00020EC3DE948E555E32F8F38A349A35AA3BA
:103DF00080EC97EFAAEBB7E38B8F9C8FAD8FBE8FD4
:103E000024EF31E040E050E02F8B388F498F5A8FFC
:103E100030E5C32E33ECD32EE12CF12C20EC422ED6
:103E20002DE9522E28E5622E25E3722E882499244E
:103E3000540133241E8A1D8A198A1A8A1B8A1C8AF5
:103E4000FFC087E396E00E94BC2E8434B9F085342D
:103E500030F48332B9F18C3209F0CCC044C08335E0
:103E600009F0C8C02F8D38A149A15AA1C901DA01B2
:103E70002C013D01882499245401E2C087E396E097
:103E800064E40E94A92B87E396E040EC5DE968E5D5
:103E900075E32AE030E00E94DD2C87E396E06CE2D7
:103EA0000E94A92B87E396E040EC57EF6AEB77E39B
:103EB0002AE030E00E94DD2C87E396E06CE20E946D
:103EC000DB2BBEC019821A821B821C821D821E82BD
:103ED0001F82188619861A861B861C861D861E86DA
:103EE0001F86188A3AC0339434E0331609F0A8C00C
:103EF00069817A818B819C8128EE33E040E050E03B
:103F00000E94892F6F8F78A389A39AA36D817E81E8
:103F10008F8198850E94892F6B8F7C8F8D8F9E8FCC
:103F200089859A85AB85BC858F8B988FA98FBA8F31
:103F30006D857E858F8598890E94892F6B017C0114
:103F400090E2C9169EE4D90690E0E90690E0F906F1
:103F500030F48CE162E30E94BA0A332471C0A0E31A
:103F6000CA16A5E7DA06A0E0EA06A0E0FA0618F409
:103F70008CE162E2F0CFB0E4CB16BCE9DB06B0E046
:103F8000EB06B0E0FB0618F48CE166E2E4CFE0E576
:103F9000CE16E3ECDE06E0E0EE06E0E0FE0618F406
:103FA0008CE162E1D8CFF0E6CF16FAEEDF06F0E062
:103FB000EF06F0E0FF0618F48CE165E1CCCF20E7D6
:103FC000C21621E1D20621E0E20620E0F20618F452
:103FD0008CE161E0C0CF30EAC31636E8D30631E0A9
:103FE000E30630E0F30618F48CE163E0B4CF8CE133
:103FF00065E0B1CF90ED292E280E49E0421500F181
:10400000032D10E0000F111F000F111F81E090E041
:104010008C0F9D1F080F191FD8016D917D918D91F7
:104020009C912AE030E040E050E00E94892F620D30
:10403000711D811D911DF8016083718382839383BB
:1040400087E396E00E94822E892B09F0FACE811434
:104050009104A104B10489F4C301B2010E94300BA0
:1040600061E070E080E090E00E94142AFFEFFE8B98
:104070001D8A198A1A8A1B8A1C8A2F89388D498DB4
:104080005A8D82169306A406B506E0F40E94DB0A58
:1040900029893A894B895C89280F311D411D511DA1
:1040A000298B3A8B4B8B5C8B3D89381708F48D8BB1
:1040B0004E89841708F48E8B0894811C911CA11CD6
:1040C000B11C56C0C301B20128EE33E040E050E01D
:1040D0000E94BB2F87E396E0BA01A9012AE030E0F5
:1040E0000E946F2C87E396E06CE20E94A92B87E385
:1040F00096E06D894AE050E00E94B72C87E396E095
:104100006CE20E94A92B69897A898B899C89A50117
:1041100094010E94BB2F87E396E0BA01A9012AE02F
:1041200030E00E946F2C87E396E06CE20E94A92B9E
:1041300087E396E06E894AE050E00E94B72C87E35F
:1041400096E06CE20E94DB2B4C0C5D1C6E1C7F1C0D
:104150008B8D9C8DAD8DBE8D84159505A605B705FF
:1041600020F44F8C58A069A07AA088249924540187
:104170002F8D38A149A15AA1285E334040405040BC
:1041800009F05ECFA296E2E10C941430AAE5B0E00B
:10419000ECECF0E20C9404308B017A018B3009F4E2
:1041A00026C18C3040F5853009F484C0863080F417
:1041B000823009F459C0833020F4813009F050C2B4
:1041C00042C0833009F461C0843009F049C265C03F
:1041D000883009F49DC0893038F4863009F486C0EF
:1041E000873009F03DC28CC0893009F499C08A300B
:1041F00009F036C2C9C0893609F482C18A3680F412
:10420000863609F42DC1873620F4853609F028C298
:104210000EC1873609F43DC1883609F021C241C17B
:104220008C3609F4C4C18D3638F48A3609F473C16A
:104230008B3609F015C2AFC18D3609F4ECC1873C4D
:1042400009F00EC200C281E069E270E00E947A11BA
:1042500000ED13E0F80181918F010E946311F3E0FA
:10426000093F1F07B9F704C282E06BE170E00E94CA
:104270007A1105EB13E0F80181918F010E9463111F
:10428000F3E0003D1F07B9F7F3C183E061E070E0A0
:104290000E947A110E941015E9C184E061E070E08B
:1042A0000E947A1181E00E9463110E945C110E94B9
:1042B000DA1EE0C16091890470E0660F771F85E027
:1042C0000E947A1100E010E008C0F801E759FB4FA6
:1042D00080810E9463110F5F1F4F8091890490E0DD
:1042E000880F991F0817190780F3C2C186E062E0A2
:1042F00070E00E947A1181E793E00E947111B8C1C9
:1043000087E061E070E00E947A1180918A04AEC17A
:1043100088E061E070E00E947A1180919B03A6C161
:1043200086E68983CE01019661E00E94C20F0E9459
:10433000790C83E080939A0368EC70E080E090E071
:104340000E94142A80919A038430E1F48FE70E943E
:10435000900A0E94A40A8983863471F489E060E29D
:1043600070E00E947A1110E00E94A40A0E9463117A
:104370001F5F1032C9F77CC189E061E070E00E94E4
:104380007A11C7C089E06DC18AE069E170E00E94DE
:104390007A1182E080939C038091A105882351F0DB
:1043A0008091A1039091A203A091A303B091A403D3
:1043B000806809C08091A1039091A203A091A303FA
:1043C000B091A4038F778093A1039093A203A0934D
:1043D000A303B093A4030CE913E0F80181918F01CA
:1043E0000E946311F3E0053B1F07B9F741C18BE061
:1043F00061E270E00E947A118091BE048F3F39F033
:104400008091BE048F5F8093BE04815002C0809172
:10441000BE040E94631110E0812F0E9499110E9436
:10442000190A0E9471111F5F1031B1F721C185E691
:1044300061E070E00E947A110932110509F015C19E
:1044400020E030E0F901E053FC4FD701A20FB31F89
:104450008C9180832F5F3F4F2932310599F759C0E6
:1044600086E661E070E00E947A110B31110509F0D7
:10447000FCC020E030E0F901EB54FC4FD701A20F63
:10448000B31F8C9180832F5F3F4F2B31310599F7FC
:1044900040C087E661E070E00E947A110E94BB167E
:1044A00038C088E661E070E00E947A1185E78A836F
:1044B000DE011396E5EBF3E08BE101900D92815064
:1044C000E1F7CE0102966CE10E94C20F0E94790CC6
:1044D00083E080939A0360E273E080E090E00E94C2
:1044E000142A80919A03843009F0BFC08FE70E949C
:1044F000900A0E94A40A8A83853509F0B6C009C0D3
:1045000089E661E070E00E947A110E944D080E94E5
:10451000920881E0ABC08AE661E070E00E947A1107
:1045200089E68E8FCE014E9661E00E94C20F0E94F6
:10453000790C83E080939A0360E273E080E090E07E
:104540000E94142A80919A03843009F08EC08FE76C
:104550000E94900A0E94A40A8E8F8E01015E1F4F56
:104560004AE3E42EF12CEC0EFD1E0E94A40AF80191
:1045700081938F01EE15FF05C1F7A5EBB3E0FE01B6
:104580007F968BE101900D928150E1F78E8D8934F9
:1045900009F06BC0BECF8BE661E070E00E947A113B
:1045A000F70180810E94E9160E94C416B2CF8CE602
:1045B00061E070E00E947A110032110571F487E623
:1045C0008AAFDE01DB96F70180E201900D92815007
:1045D000E1F7CE01CA9661E205C087E48AAFCE0159
:1045E000CA9661E00E94C20F0E94790C83E080931A
:1045F0009A036CE474E080E090E00E94142A8091B9
:104600009A03843091F58FE70E94900A0E94A40AD1
:10461000873459F57ECF8DE661E070E00E947A1113
:104620000931110511F520E030E0F901E456FC4FA5
:10463000D701A20FB31F8C9180832F5F3F4F293189
:10464000310599F766CF87EC61E070E00E947A113E
:1046500081E00E9463110E945C111092FF030AC066
:104660008AEC61E070E00E947A1180E00E946311A0
:104670000E945C11C65ADF4FE6E00C942030A0E0A7
:10468000B0E0E5E4F3E20C94003084E0A82E06E00C
:10469000B02E15E0C12E05E315E0B4E6DB2EA2E056
:1046A000EA2EF3E0FF2EA1C087E396E00E94BC2E25
:1046B000982F8093A00580919F05833021F184304D
:1046C00028F4813099F08230B8F409C0853009F4BB
:1046D00048C0853020F1863009F087C05FC0953B27
:1046E00009F083C081E080939F057FC0923609F076
:1046F0007AC0E0929F0579C090939E0590939D05A6
:10470000F0929F0572C090939B0510929C0580913A
:104710009D05892780939D05A0929F0566C0D92F8E
:10472000C0E020919B0530919C052C2B3D2B3093B4
:104730009C0520939B0580919D05892780939D056D
:10474000C0929F052536310508F44FC08CEC61E01E
:1047500070E00E947A1181E00E9463110E945C1156
:1047600042C02091990530919A05F901EB5CFA4F0E
:10477000908380919D05892780939D052F5F3F4FF2
:1047800030939A052093990580919B0590919C0503
:104790002817390750F1B0929F0527C080919D05D9
:1047A000891759F46091990570919A0580919E0539
:1047B00045E355E00E94C6200DC08BEC62E070E03E
:1047C0000E947A1180919E050E94631180910004DD
:1047D0000E946311F8018D2D11928A95E9F71092CC
:1047E0009A051092990510929F0587E396E00E9422
:1047F000822E892B09F058CFCDB7DEB7EAE00C94B2
:104800001C3081E08093FF0308C087E396E00E949C
:10481000822E892B11F00E943F238091FF03882371
:10482000A1F70895A0E0B0E0E8E1F4E20C940330D1
:104830000E94EE296115710581059105C9F30E9459
:1048400099061092D9031092DA031092DB031092AA
:10485000DC03DD24E090D903F090DA030091DB0360
:104860001091DC03102F0F2DFE2CEE240E949406D5
:104870002FEF30E040E050E00E94DD2FE60EF71E03
:10488000081F191FE092D903F092DA030093DB03AB
:104890001093DC03D39444E0D416E1F6CFEDD3E0DB
:1048A00000E010E090E1E92E97E2F92E4EC00F5F94
:1048B00019F40E944D084DC00E94940622E330E096
:1048C00040E050E00E94DD2F6F5FEFEDF3E090E0FD
:1048D00004C08191861759F39F5F9117D0F380919F
:1048E000DE0390E08E9D90018F9D300D9E9D300DDA
:1048F0001124862F90E0AC01249FC001259F900DCC
:10490000349F900D1124AA2797FDA095BA2F2091CE
:10491000D5033091D6034091D7035091D803820F2D
:10492000931FA41FB51F20919D0330919E034091BA
:104930009F035091A003281739074A075B0708F423
:10494000B6CF69931F5F183121F08881882309F061
:10495000AECFCDB7DEB7E7E00C941F301F931091B8
:1049600001041F3F09F0F1C0893409F467C08A349B
:1049700028F5883309F479C0893368F4803309F461
:1049800086C0813308F06FC08B3109F44DC081328D
:1049900009F0D5C03DC0813409F49AC0823438F49E
:1049A000893309F472C0803409F0C9C031C082343F
:1049B00009F4A1C0863409F0C2C052C0823609F49D
:1049C0009AC0833690F4883579F1893538F4823588
:1049D00009F43FC0833509F0B2C01FC08A3509F41D
:1049E000A9C0813609F0ABC073C0823791F183371B
:1049F00030F48636A9F1893609F0A1C01FC0883786
:104A000099F08A3709F496C0833709F098C005C039
:104A100087E396E069E471E019C00E94BB1687E362
:104A200096E063ED71E006C00E94C41687E396E04D
:104A30006DEE71E00E943D2D8EEF7FC00E944D080B
:104A40000E94920887E396E06CE072E00E943D2DA0
:104A500076C00E94122487E396E065E272E0F6CF0A
:104A60000E946C176CC0805368C087E396E06CEEC0
:104A700071E00E94C72B9091F803892F885F88719D
:104A8000977E892B8093F80320C089E056C087E386
:104A900096E069ED71E00E94C72B8091A10390918F
:104AA000A203A091A303B091A40320E130E040E071
:104AB00050E082279327A427B5278093A1039093E2
:104AC000A203A093A303B093A4031093010437C0DF
:104AD00087E396E063EC71E00E94C72B8091A1030D
:104AE0009091A203A091A303B091A40320E430E02D
:104AF00040E050E012C087E396E062EB71E00E9474
:104B0000C72B8091A1039091A203A091A303B09120
:104B1000A40320E230E040E050E082279327A4275E
:104B2000B5278093A1039093A203A093A303B0930E
:104B3000A40302C00E94031E8FEF809301048091A2
:104B400001048E3F09F4DDC0D4C00E9403178823FE
:104B500009F4D7C080916704882321F48FEF8093F4
:104B60000104C7C082E094E060E070E040E050E003
:104B70000E94A2069B01AC0180910104992787FD48
:104B80009095A92FB92FFC013197E930F10508F074
:104B90008CC0E753FF4F0C942F30DA01C901815CC0
:104BA0009D49A845B5438F5F9945A246B24008F09C
:104BB0007CC02093D5033093D6034093D703509302
:104BC000D8039AC02093D9033093DA034093DB03D0
:104BD0005093DC0381E0809368048EC02830310557
:104BE0004105510508F061C02093DD0385C0DA015D
:104BF000C9010197A109B1090A97A105B10508F0FA
:104C000054C02093DE0378C082E094E06DE371E04D
:104C10000E94BE0710E00EC0183130F4E12FF0E022
:104C2000E053FC4F87871F5F80E090E06DE371E009
:104C30000E94BE07009759F00E94A007009761F7F5
:104C400006C0E12FF0E0E053FC4F17861F5F1831DC
:104C5000C0F352C0253031054105510530F5209390
:104C6000F7034AC0DA01C9010197A109B109069702
:104C7000A105B105D0F48091F803887F822B809341
:104C8000F8033AC0DA01C9010197A109B1098050BE
:104C9000924CA140B04048F42093D1033093D2030A
:104CA0004093D3035093D40327C087E396E068EA88
:104CB00071E00E943D2D13C08091D9039091DA03D9
:104CC000A091DB03B091DC030196A11DB11D80937F
:104CD000D9039093DA03A093DB03B093DC030E9423
:104CE000F9168FEF8093010487E396E06AE00E9453
:104CF000DB2B0E94471E05C0809168048823E1F2E7
:104D0000EECF1F9108958FEF8093010410926804F5
:104D10000E94471E0CC087E396E00E94822E892BDA
:104D200031F087E396E00E94BC2E0E94AE24809171
:104D300001048E3F81F76AE070E080E090E00E941D
:104D4000142A04C087E396E00E94BC2E87E396E015
:104D50000E94822E892BB1F70895AAE2B0E0E3EB1E
:104D6000F6E20C94FD2F0E94E0297B018C0181E08A
:104D70000E949A0B04C087E396E00E94BC2E87E352
:104D800096E00E94822E892BB1F743982998DD2462
:104D9000D39452E6752E42E0842E912C8C0E9D1EEB
:104DA0005E010894A11CB11C33E0C32E0E94E029CF
:104DB00020E030E06E197F09800B910B693C710592
:104DC0008105910510F021E030E08D2D90E0282341
:104DD0003923232BB9F10E94E0297B018C0185B195
:104DE000846285B980ED97E00E94CF117982D40169
:104DF000E0EDF3E089E201900D928150E1F7C50109
:104E00006AE20E94C20F85B18B7D85B980E090E097
:104E10000E94CF11C0929A030E94790C62E370E065
:104E200080E090E00E94142A80919A03843051F42B
:104E3000C0929A038FE70E94900A0E94A40A8234CB
:104E400009F4DD2487E00E94122B892B79F5DD24FB
:104E5000D3942CC0439A299A85B1846285B987E39B
:104E600096E00E94BC2E8D30910569F08E30910540
:104E70001CF40A97B1F407C08332910569F08234BB
:104E8000910579F40CC087E396E064EA71E00E9432
:104E9000C72B0E94832605C00E94DA1E02C00E9412
:104EA00001244398299885B18B7D85B987E396E0E5
:104EB0000E94822E892B09F479CFCCCF8F929F92BA
:104EC000AF92BF92CF92DF92EF92FF920F931F9318
:104ED00087E00E94122B892B09F083C068EC70E0F8
:104EE00080E090E00E94142A80E090E00E94CF11C0
:104EF0000E94E0295B016C0160ECE62E62E1F62E77
:104F0000012D112DEA0CFB1C0C1D1D1D06C087E098
:104F10000E94122B892B09F062C00E94E0296E15B5
:104F20007F058007910798F387E00E94122B892B59
:104F300009F055C080ED97E00E94CF110E94E02952
:104F40007B018C0199249394882488E496E2A0E064
:104F5000B0E0A80EB91ECA1EDB1E29C0AE14BF04E5
:104F6000C006D10638F480ED97E00E94CF11882466
:104F700083941DC00E94E0296E197F09800B910B5C
:104F8000693C71058105910590F00E94E0297B0143
:104F90008C0180E0992009F481E0982E882319F48F
:104FA00080E090E002C080ED97E00E94CF1187E0A2
:104FB0000E94122B892B91F280E090E00E94CF1189
:104FC000882049F080919B038F5F83700E94E916CF
:104FD0000E94C41606C00E9412240E94BB160E94A2
:104FE000AD261F910F91FF90EF90DF90CF90BF9073
:104FF000AF909F908F90089580E06DEF77E042E052
:1050000050E00E941B290895EF92FF920F931F9387
:1050100080E00E9419080E94BA1181E161E00E94BB
:10502000732A8DE061E00E94732A89E061E00E94AA
:10503000732A8AE061E00E94732A87E060E00E94A0
:10504000732A88E060E00E94732A88E061E00E9491
:10505000DF2A0E94DA1487E396E040E052EC61E038
:1050600070E00E94FB2D0E94DC160E94C4160E9474
:10507000590D8FEF8093BE040E94FC2778940E9404
:10508000E0297B018C018091BE048F3F09F0C8C0EC
:105090000E94E0296E197F09800B910B605D7740BB
:1050A0008040904008F0BCC0EECF87E396E00E94BD
:1050B000BC2E87E396E00E94822E892BB1F787E30E
:1050C00096E062E472E00E943A2D81E793E00E944C
:1050D000731A87E396E069E572E00E943A2D87E350
:1050E00096E063E070E04AE050E00E94262D62E323
:1050F00070E080E090E00E94142A87E396E00E942E
:10510000822E04970CF187E396E00E94BC2E823435
:105110009105D1F487E396E00E94BC2E8E34910570
:1051200099F487E396E00E94BC2E8434910561F4E3
:1051300087E396E00E94BC2E819731F480E090E0F6
:105140000E94CF110E94AD264091D1035091D2030D
:105150006091D3037091D403DB01CA010197A109C7
:10516000B1090497A105B10568F44093BF04433029
:1051700029F040E052EC61E070E004C040EA56E8FB
:1051800061E070E087E396E00E94FB2D0E945E27BD
:105190004398299880E090E00E94CF110E94590D19
:1051A00080E00E949A0B8091A4040E94C50A0E948C
:1051B000790C1092290510922A0510922B0510E007
:1051C00015C062E370E080E090E00E94142A80ED58
:1051D00097E00E94CF1162E370E080E090E00E94CF
:1051E000142A80E090E00E94CF111F5F80919B0302
:1051F000811738F78091F80390E084FF09C020E020
:1052000088719070489709F421E0822F0E94F11470
:105210008FE00E9419081F910F91FF90EF90089561
:1052200080ED97E00E94CF1187E061E00E94DF2AC5
:10523000439A299A3ECF823000F5E82FF0E0EE0F36
:10524000FF1FEE55FA4F71836083882319F0813078
:10525000A1F408C0809169008C7F842B8093690041
:10526000E89A089580916900440F551F440F551F17
:10527000837F842B80936900E99A08951F920F928F
:105280000FB60F9211242F933F934F935F936F9319
:105290007F938F939F93AF93BF93EF93FF938091EF
:1052A000A2059091A305892B29F0E091A205F09128
:1052B000A3050995FF91EF91BF91AF919F918F91B8
:1052C0007F916F915F914F913F912F910F900FBE02
:1052D0000F901F9018951F920F920FB60F921124E6
:1052E0002F933F934F935F936F937F938F939F93EE
:1052F000AF93BF93EF93FF938091A4059091A50581
:10530000892B29F0E091A405F091A5050995FF915D
:10531000EF91BF91AF919F918F917F916F915F912D
:105320004F913F912F910F900FBE0F901F901895A6
:105330001F920F920FB60F9211242F933F938F93CA
:105340009F93AF93BF938091AA059091AB05A091D5
:10535000AC05B091AD053091AE050196A11DB11D12
:10536000232F2D5F2D3720F02D570196A11DB11D44
:105370002093AE058093AA059093AB05A093AC054E
:10538000B093AD058091A6059091A705A091A805C1
:10539000B091A9050196A11DB11D8093A60590931A
:1053A000A705A093A805B093A905BF91AF919F91C0
:1053B0008F913F912F910F900FBE0F901F901895D6
:1053C0008FB7F8942091AA053091AB054091AC05B8
:1053D0005091AD058FBFB901CA0108959FB7F894E8
:1053E0002091A6053091A7054091A8055091A905E7
:1053F00086B5A89B06C08F3F21F02F5F3F4F4F4FD0
:105400005F4F9FBF542F432F322F2227280F311D6C
:10541000411D511D82E0220F331F441F551F8A95E5
:10542000D1F7B901CA010895EF92FF920F931F932C
:10543000CF93DF937B018C010E94EE29EB010EC01C
:105440000E94EE296C1B7D0B685E7340C8F30894C4
:10545000E108F10801091109C851DC4FE114F10418
:105460000105110569F7CDB7DEB7E6E00C942030F1
:10547000789484B5826084BD84B5816084BD85B52F
:10548000826085BD85B5816085BDEEE6F0E08081F6
:1054900081608083E1E8F0E0108280818260808317
:1054A000808181608083E0E8F0E08081816080839A
:1054B000E1EBF0E0808184608083E0EBF0E08081CC
:1054C00081608083EAE7F0E080818460808380816E
:1054D0008260808380818160808380818068808316
:1054E0001092C1000895CF93DF93482F50E0CA0176
:1054F0008D5F934FFC0134914151544FFA018491D7
:10550000882369F190E0880F991FFC01EF52F44F56
:10551000A591B491FC01E552F44FC591D491662355
:1055200051F42FB7F8948C91932F909589238C93F5
:10553000888189230BC0623061F42FB7F8948C9175
:10554000932F909589238C938881832B88832FBFF9
:1055500006C09FB7F8948C91832B8C939FBFDF91EB
:10556000CF910895833071F0843028F48130A1F018
:10557000823021F514C08630B1F08730D1F084300C
:10558000E9F404C0809180008F7703C0809180008F
:105590008F7D80938000089584B58F7702C084B595
:1055A0008F7D84BD08958091B0008F778093B00087
:1055B00008958091B0008F7D8093B0000895FF9290
:1055C0000F931F93F62E482F50E0CA01895E934F28
:1055D000FC012491CA018D5F934FFC01149141514C
:1055E000544FFA0104910023C9F0222319F0822FAD
:1055F0000E94B22AE02FF0E0EE0FFF1FE552F44FB9
:10560000A591B4919FB7F894FF2021F48C91109547
:10561000812302C08C91812B8C939FBF1F910F918E
:10562000FF9008950F931F93482F50E0CA01895EA1
:10563000934FFC012491CA018D5F934FFC010491AB
:105640004151544FFA011491112319F420E030E034
:1056500015C0222319F0822F0E94B22A812F90E0D8
:10566000880F991F8B51944FFC01A591B4918C9197
:1056700020E030E0802311F021E030E0C9011F91EB
:105680000F910895982F8E3008F09E50977080915A
:1056900048038295880F880F807C892B80937C003B
:1056A00080917A00806480937A0080917A0086FDF0
:1056B000FCCF2091780040917900942F80E030E079
:1056C000282B392BC9010895A0E0B0E0EAE6FBE2FF
:1056D0000C9402307C016B018A01C0E0D0E00FC065
:1056E000D6016D916D01D701ED91FC910190F08192
:1056F000E02DC7010995C80FD91F015010400115B1
:10570000110571F7CE01CDB7DEB7E8E00C941E307D
:10571000EF92FF920F931F93CF93DF937C018B0146
:10572000C0E0D0E0F8010F5F1F4F6491662359F08D
:10573000D701ED91FC910190F081E02DC701099511
:10574000C80FD91FEFCFCE01CDB7DEB7E6E00C947E
:105750002030DC01ED91FC910190F081E02D099564
:105760000895EF92FF920F931F938C016DE00E94BA
:10577000A92B7C01C8016AE00E94A92B9C012E0D77
:105780003F1DC9011F910F91FF90EF900895EF9277
:10579000FF920F931F937C010E94882B8C01C701FD
:1057A0000E94B12B9C01200F311FC9011F910F9145
:1057B000FF90EF900895EF92FF920F931F937C015B
:1057C0000E94A92B8C01C7010E94B12B9C01200FC4
:1057D000311FC9011F910F91FF90EF900895CF9352
:1057E000DF93EC016115710519F420E030E00FC082
:1057F000DB010D900020E9F71197A61BB70BE8819C
:10580000F9810280F381E02DAD0109959C01C90168
:10581000DF91CF9108954F925F927F928F929F92E6
:10582000AF92BF92CF92DF92EF92FF920F931F93AE
:10583000DF93CF93CDB7DEB7A1970FB6F894DEBF55
:105840000FBECDBF2C01742ECB01223008F42AE00C
:1058500019A231E2C32ED12CCC0EDD1E822E99244A
:10586000AA24BB24672D752FA50194010E94BB2F8C
:1058700079018A01C801B701A50194010E94892F0D
:10588000472D461B0894C108D1084A3010F4405DEA
:1058900001C0495CF6014083E114F10401051105E2
:1058A00021F07E2C5F2DC801DDCFC201B6010E9420
:1058B000EF2BA1960FB6F894DEBF0FBECDBFCF91F0
:1058C000DF911F910F91FF90EF90DF90CF90BF90ED
:1058D000AF909F908F907F905F904F900895DC01E4
:1058E0002115310541F4ED91FC910190F081E02DFD
:1058F000642F099508950E940B2C0895EF92FF9252
:105900000F931F937C010E946F2C8C01C7010E9492
:10591000B12B9C01200F311FC9011F910F91FF90E6
:10592000EF900895EF92FF920F931F939A017B01DE
:1059300000E010E0B801A7010E946F2C1F910F91A9
:10594000FF90EF900895EF92FF920F931F937C01C9
:105950000E94922C8C01C7010E94B12B9C01200F48
:10596000311FC9011F910F91FF90EF900895EF92A1
:10597000FF920F931F939A01E62EFF2400E010E0A0
:10598000B801A7010E946F2C1F910F91FF90EF901B
:105990000895EF92FF920F931F937C010E94B72C02
:1059A0008C01C7010E94B12B9C01200F311FC9013E
:1059B0001F910F91FF90EF900895A0E0B0E0E3EE0B
:1059C000FCE20C940230EC016A017B0121153105E7
:1059D00041F4E881F9810190F081E02D642F09956F
:1059E0001BC02A303105B1F477FF13C06DE20E946D
:1059F000A92B8C0144275527BA014C195D096E0962
:105A00007F09CE012AE00E940B2C9C01200F311F40
:105A100004C02AE00E940B2C9C01C901CDB7DEB75F
:105A2000E8E00C941E30EF92FF920F931F937B01DE
:105A30009A010027F7FC0095102FB801A7010E94DA
:105A4000DD2C1F910F91FF90EF900895EF92FF9240
:105A50000F931F937C010E94132D8C01C7010E949C
:105A6000B12B9C01200F311FC9011F910F91FF9095
:105A7000EF9008950E94EF2B0895EF92FF920F93FD
:105A80001F937C010E943A2D8C01C7010E94B12B0B
:105A90009C01200F311FC9011F910F91FF90EF90C2
:105AA000089508951F920F920FB60F9211242F930D
:105AB0003F934F938F939F93EF93FF938091C000F9
:105AC00082FD1DC04091C6002091EF053091F00588
:105AD0002F5F3F4F2F7330708091F1059091F20549
:105AE0002817390771F0E091EF05F091F005E155C5
:105AF000FA4F40833093F0052093EF0502C0809168
:105B0000C600FF91EF919F918F914F913F912F91FF
:105B10000F900FBE0F901F9018951F920F920FB607
:105B20000F9211242F933F938F939F93EF93FF93A3
:105B300020913306309134068091350690913606D7
:105B40002817390731F48091C1008F7D8093C100FF
:105B500014C0E0913506F0913606ED50FA4F2081E1
:105B6000809135069091360601968F7390709093D0
:105B70003606809335062093C600FF91EF919F91E2
:105B80008F913F912F910F900FBE0F901F901895FE
:105B9000A0E0B0E0EEECFDE20C94FE2FFC011382DD
:105BA000128288EE93E0A0E0B0E084839583A68320
:105BB000B7838BE893E091838083758764875787E9
:105BC0004687318B208B138B028BF58AE48AD78A28
:105BD000C68AB18EA08E938E828E8F85848F88899F
:105BE000858F8989868F8A89878F8B8980A3209664
:105BF000ECE00C941A30AF92BF92DF92EF92FF92DA
:105C00000F931F93CF93DF93EC017A018B01DD2477
:105C1000403081EE580780E0680780E0780711F097
:105C2000DD24D39491E0A92EB12CEC89FD89DD20EF
:105C300069F0C50108A002C0880F991F0A94E2F715
:105C4000808360E079E08DE390E005C0108260E839
:105C500074E88EE190E0A80197010E94BB2F2150CB
:105C6000304040405040569547953795279580E104
:105C70002030380720F0DD2011F0DD24D6CFE88970
:105C8000F9893083EA89FB89208319A2EE89FF898B
:105C9000408121E030E0C9010C8C02C0880F991FBF
:105CA0000A94E2F7482B4083EE89FF894081C901BD
:105CB0000D8C02C0880F991F0A94E2F7482B40838D
:105CC000EE89FF894081C9010E8C02C0880F991F9F
:105CD0000A94E2F7482B4083EE89FF8980810F8C7C
:105CE00002C0220F331F0A94E2F720952823208355
:105CF000DF91CF911F910F91FF90EF90DF90BF90B8
:105D0000AF900895DC011C96ED91FC911D97E05C2D
:105D1000FF4F2191319180819181281B390B2F7385
:105D20003070C901089587E396E00E94822E892B86
:105D300011F00E94512D0895DC011C96ED91FC910B
:105D40001D97E05CFF4F20813181E054F040DF017E
:105D5000AE5BBF4F8D919C9111972817390719F4AD
:105D60002FEF3FEF07C08D919C91E80FF91F8081C5
:105D7000282F30E0C9010895DC011C96ED91FC91BB
:105D80001D97E05CFF4F20813181E054F040DF013E
:105D9000AE5BBF4F8D919C9111972817390719F46D
:105DA0002FEF3FEF10C08D919C911197E80FF91FD5
:105DB00020818D919C91119701968F73907011960F
:105DC0009C938E9330E0C9010895DC0191968C91EB
:105DD0009197882339F05496ED91FC9155978081E5
:105DE00086FFF9CF91961C920895CF93DF93EC0133
:105DF000EE85FF85E05CFF4F20813181E054F0406B
:105E00002F5F3F4F2F733070DF01AE5BBF4F8D911F
:105E10009C91119728173907D1F3E05CFF4F8081DF
:105E20009181E054F040E80FF91F6083EE85FF8513
:105E3000E05CFF4F31832083EE89FF89208181E080
:105E400090E00F8C02C0880F991F0A94E2F7282B6C
:105E5000208381E089A3EC89FD898081806480832F
:105E600081E090E0DF91CF9108958F929F92AF9261
:105E7000BF92CF92DF92EF92FF920F931F9300D0C9
:105E800000D00F92EDB7FEB7319684E0ADB7BEB744
:105E900011968C9383E0818387E0828385E08383FE
:105EA00081E0848387E396E06FEA75E043EF55E095
:105EB00025EC30E004EC10E0B0ECEB2EF12CA1EC82
:105EC000CA2ED12CF2ECAF2EB12CE6EC8E2E912CFA
:105ED0000E94C82D0F900F900F900F900F901F9160
:105EE0000F91FF90EF90DF90CF90BF90AF909F9079
:105EF0008F900895CF93DF930E94382A0E94042840
:105F0000C3E9DEE20E9408122097E1F30E94932E7B
:105F1000F9CF629FD001739FF001829FE00DF11DC8
:105F2000649FE00DF11D929FF00D839FF00D749F13
:105F3000F00D659FF00D9927729FB00DE11DF91FBF
:105F4000639FB00DE11DF91FBD01CF01112408951C
:105F500097FB092E07260AD077FD04D086D006D0FD
:105F600000201AF4709561957F4F0895F6F790958B
:105F700081959F4F0895A1E21A2EAA1BBB1BFD011C
:105F80000DC0AA1FBB1FEE1FFF1FA217B307E40718
:105F9000F50720F0A21BB30BE40BF50B661F771F70
:105FA000881F991F1A9469F7609570958095909550
:105FB0009B01AC01BD01CF01089597FB092E052679
:105FC0000ED057FD04D0D7DF0AD0001C38F450950E
:105FD0004095309521953F4F4F4F5F4F0895F6F70D
:105FE00090958095709561957F4F8F4F9F4F089545
:105FF0002F923F924F925F926F927F928F929F92D9
:10600000AF92BF92CF92DF92EF92FF920F931F93C6
:10601000CF93DF93CDB7DEB7CA1BDB0B0FB6F89477
:10602000DEBF0FBECDBF09942A88398848885F84B7
:106030006E847D848C849B84AA84B984C884DF8028
:10604000EE80FD800C811B81AA81B981CE0FD11D0C
:106050000FB6F894DEBF0FBECDBFED010895EE0F71
:10606000FF1F0590F491E02D0994AA1BBB1B51E181
:1060700007C0AA1FBB1FA617B70710F0A61BB70BB8
:10608000881F991F5A95A9F780959095BC01CD015D
:106090000895911106C0803219F089508550D0F7CB
:0C60A0000895992788270895F894FFCFF1
:1060AC004E6F005965730054582074696D656F7597
:1060BC007421006D6F64756C65206C6F636B656427
:1060CC003F00486F70206368616E6E656C20002025
:1060DC0040200053004E2F4100386368002C002CE8
:1060EC00205B005D20280029004E4F5420454E4176
:1060FC00424C45440053656E64696E672073657449
:10610C0074696E677320746F2052580A005265735D
:10611C00657474696E672073657474696E67732037
:10612C006F6E2052580A0041626F7274656420656C
:10613C00646974730A00696E76616C6964207365B6
:10614C006C656374696F6E000D0A496E76616C69DB
:10615C006420696E707574202D206469736361729C
:10616C006465642107007363616E6E6572206D6FE8
:10617C0064650053657474696E677320736176652A
:10618C006420746F20454550524F4D0A005265767D
:10619C0065727465642073657474696E67732066C8
:1061AC00726F6D20454550524F4D0A004C6F616423
:1061BC00656420666163746F7279206465666175CD
:1061CC006C74730A004B657920616E64206368619E
:1061DC006E6E656C732072616E646F6D697A656446
:1061EC000A004F70656E4C52536E672054582073E2
:1061FC0074617274696E672000206F6E204857209E
:10620C000050504D005253534900534441005343E6
:10621C004C00525844005458440041494E004C42E2
:10622C004545500053504B54524D0053425553006A
:10623C0053554D44004C4C494E440000342B340013
:10624C003800382B340031320031322B34003136E7
:10625C000001000000C01200001A400AA1204EA547
:10626C00001B1E27522C23308025000005400AA15C
:10627C00204EA50020244EA52C2330004B000006F8
:10628C00400AD0009D49007B289D492C233000E119
:10629C00000005400A4501D7DC03B81E0EBF0023E1
:1062AC002E48E801008A400A6001555502AD1E20B7
:1062BC00000023C88025000005400AA1204EA5003F
:1062CC0020244EA52C233000020002000200020004
:1062DC0002000200020002000200020002000200A2
:1062EC0002000200020002FF01610265026A026EF6
:1062FC0002720276027A027E0284028B029002956E
:10630C00029B029B029B029B0235019C02A002A2F3
:10631C0002A602A902AE02350100070B0C101115E2
:10632C0000160A1322312900000000F52E642B827E
:08633C002EBC2E9C2EE52E0064
:107E00000F92CDB7DEB7112484B714BE81FFF1D035
:107E100082E08093C00088E18093C10086E0809377
:107E2000C20080E18093C4008EE0CDD088249924E4
:107E3000CC24C394F5E0DF2EE1E1EE2E73E0F72EC3
:107E4000B6D0082F813479F4B2D08983C2D0898129
:107E5000823811F481E005C0813811F485E001C059
:107E600083E09ED09AC0823411F484E103C085344B
:107E700019F485E0B6D091C0853561F498D0082F0B
:107E800010E095D090E0982E8824802A912A880CC2
:107E9000991C82C0863521F484E0A3D080E0E1CF34
:107EA000843609F04CC083D082D0A82E80D0B82E62
:107EB00000E011E07CD0F80181938F01AE16D1F77C
:107EC00088D0FB2DF53489F4E0E0F1E00BC0F9999E
:107ED000FECF92BC81BC0894811C911C819180BD15
:107EE000FA9AF99AEA1598F358C08B2D863409F05E
:107EF00054C0F401F7BEE89507B600FCFDCFF401CD
:107F0000A0E0B1E02C9130E011968C91119790E0B7
:107F1000982F8827822B932B12960C01C7BEE895C9
:107F20001124329681E0A038B80761F7F401D7BE7A
:107F3000E89507B600FCFDCFE7BEE8952EC0843774
:107F4000F1F435D034D0182F32D0B82E42D0FB2DDA
:107F5000F63421F4F40105914F010CC0FB2DF534EA
:107F600049F4F999FECF92BC81BC0894811C911C04
:107F7000F89A00B5802F14D0115049F70EC08537FC
:107F800039F427D08EE10CD085E90AD08FE069CF93
:107F9000813511F488E017D01CD080E101D050CF9A
:107FA0009091C00095FFFCCF8093C600089580910A
:107FB000C00087FFFCCF8091C00084FD01C0A89560
:107FC0008091C6000895E0E6F0E098E19083808318
:107FD0000895EDDF803219F088E0F5DFFFCF84E10E
:107FE000DFCF1F93182FE3DF1150E9F7F2DF1F9166
:0E7FF0000895282E80E0E7DFEE27FF27099492
:027FFE0001057B
:0400000300007E007B
:00000001FF
